:10000000831610308500860183120C308500013084
:1000100086000C308C0001308D000C308E000030DA
:100020008F007D20141841280C308C0000308D008A
:1000300004308E0000308F007D20141841280430D9
:100040008C0000308D0000308E0001308F007D204C
:100050001418412800308C0001308D0008308E00CB
:1000600001308F007D201418412808308C000130A9
:100070008D000C308E0000308F007D201418412838
:100080001428A120051E412894018501860105142C
:10009000A120A120A120A12005101E30950005114E
:1000A000AF200515AF20950B4F281E309500851108
:1000B000AF208515AF20950B57280F3095000610FF
:1000C000AF200614AF20950B5F283C30950006103A
:1000D000A120A120A1200614A120A120950B672812
:1000E0000430930085018601AF200D30850001307A
:1000F0008600AF20930B72280928FF3090009101F1
:10010000910A9401043093000C0885000D088600C4
:1001100010089200051E9F28920B8A280E08850061
:100120000F08860011089200051E9F28920B942844
:10013000930B8428900B9D280800910A8228940A2A
:100140000800F4309000FF3091000000910BA528CA
:10015000900BA3282C309000900BAC2808000A309C
:10016000920000000000A120920BB12800000000C6
:0801700000000000000008007F
:02400E00F23F7F
:00000001FF
